:020000040800F2
:10000000001000207D150008C5150008C515000862
:10001000C5150008C5150008C5150008000000003A
:10002000000000000000000000000000C5150008EE
:10003000C515000800000000C5150008C51500081A
:1000400000000000000000000000000000000000B0
:1000500000000000000000000000000000000000A0
:100060000000000000000000000000000000000090
:100070000000000000000000000000000000000080
:100080000000000000000000000000000000000070
:100090000000000000000000000000000000000060
:1000A0000000000000000000000000000000000050
:1000B0000000000000000000000000000000000040
:1000C0000000000000000000000000000000000030
:1000D0000000000000000000000000000000000020
:1000E0000000000000000000000000000000000010
:1000F0000000000000000000000000000000000000
:1001000000000000000000000000000000000000EF
:1001100000000000000000000000000000000000DF
:1001200000000000000000000000000000000000CF
:1001300000000000000000000000000000000000BF
:1001400000000000000000000000000000000000AF
:10015000000000000000000000000000000000009F
:10016000000000000000000000000000000000008F
:10017000000000000000000000000000000000007F
:08018000000000000000000077
:100188000448054B10B5834203D0044B002B00D024
:10019800984710BD1402002014020020000000003F
:1001A80006480749091A8B10C90FC91810B5491014
:1001B80003D0044B002B00D0984710BD1402002038
:1001C800140200200000000010B5074C2378002B13
:1001D80009D1FFF7D5FF054B002B02D0044800E0FA
:1001E80000BF0123237010BD14020020000000008E
:1001F800C8150008054B10B5002B03D00449054865
:1002080000E000BFFFF7CCFF10BDC04600000000B3
:1002180018020020C815000802B4714649084900B0
:10022800095C49008E4402BC7047C046002243085E
:100238008B4274D303098B425FD3030A8B4244D3A6
:10024800030B8B4228D3030C8B420DD3FF220902E8
:1002580012BA030C8B4202D31212090265D0030BA7
:100268008B4219D300E0090AC30B8B4201D3CB039D
:10027800C01A5241830B8B4201D38B03C01A5241DF
:10028800430B8B4201D34B03C01A5241030B8B42E1
:1002980001D30B03C01A5241C30A8B4201D3CB02CC
:1002A800C01A5241830A8B4201D38B02C01A5241B1
:1002B800430A8B4201D34B02C01A5241030A8B42B4
:1002C80001D30B02C01A5241CDD2C3098B4201D3CC
:1002D800CB01C01A524183098B4201D38B01C01A4A
:1002E800524143098B4201D34B01C01A52410309C1
:1002F8008B4201D30B01C01A5241C3088B4201D370
:10030800CB00C01A524183088B4201D38B00C01A1C
:10031800524143088B4201D34B00C01A5241411A43
:1003280000D20146524110467047FFE701B5002050
:1003380000F006F802BDC0460029F7D076E77047FE
:100348007047C04670B50C4D0C4E761BB61005D0E4
:10035800002408CD01349847A642FAD101F030F9BB
:10036800074D084E761BB61005D0002408CD013481
:100378009847A642FAD170BD041600080416000872
:100388000416000808160008F0B5C64600B50F2A7E
:1003980043D90B00032603431E400C000300002E24
:1003A80040D11500103D2D09AC462D01A8468044CA
:1003B80000E03B00676825685F60E7681D60DF60F4
:1003C8001F00A56810379D6010344345F1D165467C
:1003D8000F230C2401352D014919134045191442E6
:1003E80023D08C59AC5104369C1B032CF9D8032418
:1003F800043B9B0801339B002240ED18C918561E88
:10040800002A07D0002300E02300CA5C5C1CEA54E1
:100418009E42F9D104BC9046F0BD0500561E002A44
:10042800F0D1F7E7561E0500ECE71A00F6E7C046DC
:10043800002070470278437812021343014A0020D3
:10044800138070470000002010B501F092F80020DA
:1004580010BD10B501F083F8002010BD10B50400E0
:1004680001F085F800F03EFA200001F07CF800F079
:1004780041FA200001F07CF822001021722000F0DF
:10048800E9F8002010BD000070B50400002501F057
:100498006EF80B4B1B88AB4209D8200001F068F8B6
:1004A80022001021722000F0D5F8002070BD00F065
:1004B80019FA200001F057F8013500F01BFAE8E7B7
:1004C800000000201FB5102222496846FFF75CFF94
:1004D80000F078F900F0A2F900F0E0F901F03EF838
:1004E800684601F03CF8682000F024FA652000F026
:1004F80021FA582000F01EFA582000F01BFA582064
:1005080000F018FA0A2000F015FA00F08BF8102114
:10051800114A6B2000F080F81021104A702000F07A
:100528007BF800210E4A782000F076F8012312218A
:100538000C4A6D2000F058F802210B4A732000F095
:100548006BF810216620094A00F066F800F0D4F82C
:10055800FCE7C046F31500085B04000865040008C2
:1005680039040008510400083D04000891040008FB
:100578000120704770B50024844201DB00201FE091
:100588004D780B782E00303EF6B2092E0CD8165551
:100598001D00303DEEB2092E15D8135D2D011D4307
:1005A800155501340231E7E72E00413E052E02D8E9
:1005B800373D1555ECE72E00613E052E01D9012087
:1005C80070BD573DF5E71D00413D052D05D8373B6A
:1005D800155D1B012B431355E3E71D00613D052DF8
:1005E800EDD8573BF4E70000F0B5094E0500346834
:1005F80001200F2C0BDCBF2909D8064827013D54E0
:10060800C019416082600373002001343460F0BD7A
:10061800300200203402002010B50023FFF7E4FF69
:1006280010BD000010B50021074A7620FFF7F4FF3F
:100638000021064A7720FFF7EFFF00217920044ABE
:10064800FFF7EAFF10BDC04679050008B1060008AB
:1006580095060008F8B50D0014000F2700F06AF998
:100668006519AC4203D10A2000F064F9F8BD23787B
:10067800054E1B09F05C00F05DF9237801343B401E
:10068800F05C00F057F9ECE7E015000807B56B4699
:10069800DA1D044B72201B6801211370FFF7DAFF83
:1006A80000200EBD300200200322114BF0B5944605
:1006B8001C6800230F4D8DB0E6B2B34209DB6146DA
:1006C80061436A467220C9B2FFF7C4FF00200DB02B
:1006D800F0BD624669465A431801475D28188F5491
:1006E8004168007B6A44013351709070DBB2E4E7E3
:1006F8003002002034020020F0B52F4CA54400F051
:1007080001F92E4B2E491A6800239A4204DC07D1BE
:1007180093239B009D44F0BD1C010C5D84423FD196
:100728000127274D1C012E19337B3B4218D000238B
:100738006A46137200F0E6F8C8226B469B181870D8
:1007480000F0E0F8C9226B469B18187002AA38001E
:1007580032A9FFF70FFF0028DAD16B461B7A7360C6
:1007680000262B195B685B00B3421BD800F0CAF85F
:100778000A2801D00D28CBD12C19656802AA2800B7
:1007880032A9FFF7F7FE0028C2D1E9B2A36802A890
:10079800984701AA107001217A20FFF75BFFB7E79D
:1007A8000133B2E700F0AEF80A28B1D00D28AFD077
:1007B80032ABF0540136D4E7B4FDFFFF300200201D
:1007C80034020020F0B590270024012503260423D5
:1007D80097B0FF05380005A9059306950794089674
:1007E80000F02AFB102305A9380005930695079405
:1007F800089600F021FB05230AA80B930A960D948E
:10080800139400F0ADF80723210001A80193029585
:100818000394049400F086FA17B0F0BD802170B5F7
:100828001B4C8902626988B00A436261636990203F
:100838000B400193019BC023DB0001250326039392
:10084800022303A9C005049305950795069600F0B1
:10085800F3FA8021A269C9010A43A261A3690D487C
:100868000B400293029B236BB3431D430A4B256342
:10087800036096231B02436000238360C360036107
:1008880083610C33436100F041FC08B070BDC04681
:100898000010024000040020003801408020104A67
:1008A80070B55169800201435161536986B00340B4
:1008B80000939024009B012380250026E405200056
:1008C800029301A9023304930195039600F0B4FA48
:1008D80032002900200000F061FB06B070BDC04660
:1008E80000100240902010B501228021C00500F0C0
:1008F80055FB10BD902010B500228021C00500F0E6
:100908004DFB10BD37B508256B46DC1D012232238F
:100918002100064800F02CFC002801D120783EBDBB
:10092800034A136A2B431362EEE7C0460004002013
:100938000038014007B56B460122D91D0870024BEB
:10094800024800F08DFC07BD881300000004002059
:10095800024B1868421C1A607047C04634030020D6
:10096800F0B50368050085B0DB072FD42B689B071B
:1009780000D581E02B681B0700D5BCE02B685B071E
:1009880000D5DFE02B68DB061AD56A690423B54C6D
:10099800012A00D04AE1616B02270B436363636B52
:1009A8001A436263FFF7D4FF0600636B3B4200D132
:1009B80035E1F821626BAB698A43DB00134363635B
:1009C800296A002900D059E1002013E00C21A54C28
:1009D80062680A40042A06D063680B40082B0BD1D2
:1009E8006368DB0308D523689B03BFD56B68002BBE
:1009F800BCD1012005B0F0BD6B68012B13D1802359
:100A080022685B0213432360FFF7A2FF80270600DA
:100A1800BF0223683B42A9D1FFF79AFF801B6428D5
:100A2800F7D90320E6E7002B16D123688E4A8027E2
:100A38001340236023688D4ABF0213402360FFF7E9
:100A480087FF060023683B4200D18FE7FFF780FF4E
:100A5800801B6428F6D9E4E7052B05D1802322689A
:100A6800DB0213432360CAE723687F4A13402360ED
:100A780023687E4A1340C6E70C227A4C6368134207
:100A880006D063681340082B10D16368DB030DD4CC
:100A980023689B0702D5EB68012BAAD1F8212268AD
:100AA8002B698A43DB001343236063E7EA68012369
:100AB800002A0FD02268022713432360FFF748FF5C
:100AC800060023683B42E9D1FFF742FF801B02285A
:100AD800F7D9A6E7226802279A432260FFF738FF72
:100AE800060023683B4200D144E7FFF731FF801B33
:100AF8000228F6D995E7EA6901235A4C002A10D052
:100B0800626A022713436362FFF722FF0600636AE3
:100B18003B4200D032E7FFF71BFF801B0228F6D9C3
:100B28007FE7626A02279A436262FFF711FF0600B5
:100B3800636A3B4200D121E7FFF70AFF801B0228C6
:100B4800F6D96EE780220021464C5205E3690091F0
:100B5800134208D1E3691343E361E3691340039344
:100B6800039B012300938027414E7F0033683B425B
:100B780006D0AB68012B13D1226A1343236230E0FD
:100B880033683B433360FFF7E3FE019033683B4231
:100B9800EFD1FFF7DDFE019BC01A6428F6D940E7C4
:100BA8000122002B14D1236A022793432362236A6C
:100BB800033293432362FFF7CBFE0600236A3B42CE
:100BC80016D0FFF7C5FE2B4B801B9842F6D928E7B5
:100BD800052B16D1216A013B0B432362236A1A4372
:100BE8002262FFF7B5FE02270600236A3B420FD0B8
:100BF800009B012B00D0C5E6E3691F4A1340E3615F
:100C0800C0E6236A934304222362236A9343B5E729
:100C1800FFF79EFE174B801B9842E6D901E7FFF7C6
:100C280097FE801B022800D8BFE6FAE6053203D1FA
:100C3800626B9A436263BCE6626B0227134301222C
:100C48006363636B93436363FFF782FE0600636B22
:100C58003B4200D1B4E6FFF77BFE801B0228F6D9A1
:100C6800DFE6C04600100240FFFFFEFFFFFFFBFF6C
:100C78000070004088130000FFFFFFEF0C22264C95
:100C8800012063681340082B00D1B3E62368234A88
:100C98001340236002292FD1FFF75AFE8027060050
:100CA800BF0423683B4221D10F22E36A8026934385
:100CB800EA6AB6041343E362696AAB6A62680B4383
:100CC80017490A4013436360802322685B04134377
:100CD8002360FFF73DFE05002368334200D073E62A
:100CE800FFF736FE401B0228F6D99AE6FFF730FEDA
:100CF800801B0228D5D994E6FFF72AFE8026050036
:100D0800B6042368334200D15EE6FFF721FE401B9C
:100D18000228F6D985E6C04600100240FFFFFFFE14
:100D2800FFFFC2FFF7B501223E4C050023680F0004
:100D380013408B4212D32A68930719D4D3071FD4C0
:100D4800012322681A40BA425DD82B685B0761D438
:100D5800E122354BD20300201A6008E02368934350
:100D68000B432360236813408B42E4D00120FEBD6F
:100D7800F0202E494B688343A86803434B60DDE7A6
:100D88002A4E6A683368012A1AD19B03EED50321DB
:100D980073688B4313437360FFF7DAFD6B68019048
:100DA800012B15D10C2273681340042BC8D0FFF710
:100DB800CFFD019BC01A1E4B9842F3D90320D6E7FA
:100DC800022A02D19B01E2D4D0E79B07DFD4CDE70A
:100DD800022B12D00C2273681342B1D0FFF7B8FD72
:100DE800019BC01A124B9842F4D9E7E7FFF7B0FD10
:100DF800019BC01A0E4B9842E0D80C22736813402E
:100E0800082BF3D19CE722689A43226022681A4291
:100E18009BD0ABE7054A074953680B40E9680B4389
:100E2800536095E7002002400400002000100240B3
:100E380088130000FFF8FFFF0023F0B587B00A68A9
:100E48001400DC4001D107B0F0BD012614009E401B
:100E580034400294324200D192E04A68150001926F
:100E6800102295430395022D0DD107240F251C4010
:100E7800A400A540DA0892008218176AAF430D69EA
:100E8800A5402F43176203225C00A240D543AC461D
:100E9800032507689743019A2A40A240039D3A43D5
:100EA800013D0260012D0FD8624685681540CA6869
:100EB800A2402A4382604568019AB5430126120977
:100EC80032409A402A4342606546C2682A408D688B
:100ED800A54080242A43C260019A640522424FD06B
:100EE80001250F27274A94692C43946192699C082D
:100EF8002A4002351D40AD00AF400592059A224AAE
:100F0800A400A418A6680022BE439027FF05B84293
:100F18000CD01E4F0132B84208D01D4F0132B842E2
:100F280004D01C4F0132B84200D00232AA403243EA
:100F3800A260194A029C1668029D019FE44335434A
:100F4800FF0301D43500254015605668029D019FB6
:100F58003543BF0301D43500254055609668029D8E
:100F6800019F3543FF0201D4350025409560D568BF
:100F7800029E019F2E43BF0201D425402E00D66059
:100F880001335CE700100240000001400004004803
:100F980000080048000C004800040140002A01D065
:100FA800816170478162FCE7F8B504000D00170005
:100FB8001E002268D3692B405B1B59424B41BB4240
:100FC80001D0002018E0069B0133F3D0069B002BCC
:100FD80013D123680C491A6803200A401A609A68DA
:100FE800A331FF318A439A602200202369321370AB
:100FF8005370002368342370F8BDFFF7A9FC069BE3
:10100800801B9842D5D9E4E75FFEFFFF030070B567
:101018009A681D6904682A435D69C1692A43206882
:10102800334D0A43284002432260626831481D6AF2
:101038000240D868024362609A69A0682A432E4D2C
:101048002840024303208025A2602C4A2D02126BFF
:101058000240013A022A43D82948805CA94220D19B
:1010680008281BD8FFF7D8F83E1A051A3E1A1A1A8C
:1010780015005968234B4808C018FFF7D7F883B202
:10108800002019000F221B0791435B0F0B43E360FD
:1010980070BD5968802348085B02EDE701200023F2
:1010A800EFE708281AD8FFF7B7F80F1905190F192D
:1010B800191914005968144B4808C018FFF7B6F8F6
:1010C80080B2E0600020E3E75968E1234808DB03C9
:1010D800F3E75968802348081B02EEE70120D7E7A9
:1010E800A942F1D15968E12348081B04C4E7C04666
:1010F800F369FFFFFFCFFFFFFFF4FFFF001002407F
:10110800F01500080048E8010024F40070B5041E3A
:1011180001D1012070BD050069352B78DAB2002BAA
:1011280002D1030068331A70242301262B70226829
:1011380020001368B3431360FFF768FFB042E8D09C
:1011480023680A495A6800200A4008215A609A68A8
:101158008A439A601A68164322001E602023E066BC
:101168006A3268342B7013702070D3E7FFF7FFFFE3
:10117800F0B585B0039303006A3317001A780400AA
:101188000D000220202A39D10138002936D0002F3D
:1011980034D08022A1685201914204D12269002AE8
:1011A80001D105422AD12200683211780220012992
:1011B80024D0012111700022E26622321A70FFF752
:1011C800C7FB23008021A26858331F805F80060078
:1011D800490104338A4215D12269002A10D11F4AD5
:1011E8001A801F8822005A32138898B2002B10D117
:1011F800230020226A3368341A70207005B0F0BDCD
:10120800FF22EDE7002AECD12269002AF8D07F22DC
:10121800E6E713882021013B9BB21380039B002241
:10122800009320003300FFF7BFFE002813D1A26807
:101238002368110080225201914207D12269002AB5
:1012480004D19B8C3B402B800235CBE79B8C3B40E9
:101258002B700135C6E70320D0E7C046FF01000028
:10126800F0B585B003930300693302931B7804003B
:101278000D0016000220202B48D10138002945D046
:10128800002A43D08023A2685B019A4204D12369D3
:10129800002B01D1014239D1230068331A7802208A
:1012A800012A33D001221A700023029AE3662133FF
:1012B8001370FFF74DFB230050331E805E8080269D
:1012C80007007601210052310B889AB2002B0ED10B
:1012D800039B4021009320003B00FFF765FE002898
:1012E80013D12023029A6834137020700EE00B8803
:1012F8000022013B9BB20B80039B802100932000BE
:101308003B00FFF751FE002802D0032005B0F0BDD6
:10131800A3682268B34208D12369002B05D12B8822
:101328000235DB05DB0D1385CCE72B7801351385FA
:10133800C8E70000224BF7B51B68224A18001100C5
:1013480010301C780C705C784C709C788C70DC7851
:101358000433CC7004318342F3D104211A4801AB21
:10136800160000240C36375DE7540134042CFAD1FA
:10137800013C21420FD19D781E78455D865D5C78E1
:101388005D70124DDF78DE708E08045DAE5DC75D5E
:1013980074409F701C7014781E7801317440147466
:1013A8005E785478744054749E7894787440947439
:1013B800DE78D47804327440D4732C29D0D1F7BDA8
:1013C80038030020500300201301002008000020EB
:1013D8000B4B70B55B680B4A1D0000018018103577
:1013E800190000220C78865C013274400C700131BF
:1013F800042AF7D104330430AB42F1D170BDC046A2
:101408003803002050030020094B10B559680948DB
:101418000A00143110321300103B1C78045D1C7054
:1014280004339342F9D15A1C8A42F4D110BDC04604
:1014380038030020130100200D4B5B6859795A7856
:101448005970597A5971597B5A735972997A9A789D
:101458009970997B9A729A799971D97B9A73DA788B
:10146800D970D97AD973D979DA71D9727047C046E7
:1014780038030020C20903001B2050435B0058407A
:10148800C0B27047F0B5002087B0FFF7A1FF012573
:10149800FFF7BAFFFFF7D0FF214B5C68230010333A
:1014A80005932378E778019301986378584002936D
:1014B800A37803937B401E0004934640FFF7DAFFAE
:1014C800019B58407040039B207002985840FFF7DA
:1014D800D1FF029B5840704060700498FFF7CAFF24
:1014E800039B58407040A07001987840FFF7C2FFF6
:1014F80078404640059BE67004349C42D1D12800D0
:101508000135EDB2FFF764FF0A2DC1D1FFF77CFF6B
:10151800FFF792FF2800FFF75BFF07B0F0BDC0465A
:10152800380300200023CA5CC2540133102BFAD1BF
:101538007047000010B5024B1860FFF7FBFE10BDA6
:1015480038030020010010B5034841600830FFF758
:10155800E9FFFFF797FF10BD38030020704710B56B
:10156800FFF7E8FF10BD10B5FFF7ECFF10BD70479F
:1015780070477047002103E00B4B5B584350043120
:101588000A480B4B42189A42F6D30A4A02E0002353
:1015980013600432084B9A42F9D300E000BFFEF70B
:1015A800D1FEFEF78FFFFEE70C16000800000020B2
:1015B800140200201402002070040020FEE700003E
:1015C800F8B5C046F8BC08BC9E467047F8B5C0469A
:0815D800F8BC08BC9E467047F8
:1015E0003031323334353637383941424344454659
:1015F0000408022B7E151628AED2A6ABF715880973
:04160000CF4F3C008C
:04160400FD010008DC
:04160800D101000804
:10160C000A00000000127A008D010204081020402C
:10161C00801B3652096AD53036A538BF40A39E814F
:10162C00F3D7FB7CE339829B2FFF87348E4344C472
:10163C00DEE9CB547B9432A6C2233DEE4C950B4293
:10164C00FAC34E082EA16628D924B2765BA2496D46
:10165C008BD12572F8F66486689816D4A45CCC5DA0
:10166C0065B6926C704850FDEDB9DA5E154657A719
:10167C008D9D8490D8AB008CBCD30AF7E45805B888
:10168C00B34506D02C1E8FCA3F0F02C1AFBD03015C
:10169C00138A6B3A9111414F67DCEA97F2CFCEF087
:1016AC00B4E67396AC7422E7AD3585E2F937E81CE5
:1016BC0075DF6E47F11A711D29C5896FB7620EAAC5
:1016CC0018BE1BFC563E4BC6D279209ADBC0FE7866
:1016DC00CD5AF41FDDA8338807C731B11210592732
:1016EC0080EC5F60517FA919B54A0D2DE57A9F9367
:1016FC00C99CEFA0E03B4DAE2AF5B0C8EBBB3C83D8
:10170C00539961172B047EBA77D626E16914635579
:10171C00210C7D637C777BF26B6FC53001672BFEF0
:10172C00D7AB76CA82C97DFA5947F0ADD4A2AF9C2B
:10173C00A472C0B7FD9326363FF7CC34A5E5F17102
:10174C00D8311504C723C31896059A071280E2EB0B
:10175C0027B27509832C1A1B6E5AA0523BD6B3299B
:10176C00E32F8453D100ED20FCB15B6ACBBE394A28
:10177C004C58CFD0EFAAFB434D338545F9027F502F
:10178C003C9FA851A3408F929D38F5BCB6DA21102E
:10179C00FFF3D2CD0C13EC5F974417C4A77E3D64C6
:1017AC005D197360814FDC222A908846EEB814DEF6
:1017BC005E0BDBE0323A0A4906245CC2D3AC629180
:1017CC0095E479E7C8376D8DD54EA96C56F4EA656A
:1017DC007AAE08BA78252E1CA6B4C6E8DD741F4B69
:1017EC00BD8B8A703EB5664803F60E613557B986D7
:1017FC00C11D9EE1F8981169D98E949B1E87E9CE84
:10180C005528DF8CA1890DBFE6426841992D0FB098
:04181C0054BB1600A3
:040000050800157D5D
:00000001FF
